:0300000002405C5F
:0C405C0078FFE4F6D8FD75816A0240A3ED
:10152C0020000A3C2E2E2E3E004950436F6E6E65F5
:10153C0063745245510A004950436F6E6E65637473
:10154C00000A49504E6F41434B210A003E432C5632
:10155C002C52432CC0E4E0EFF2E5F020D1E8EDEAA8
:10156C00EEEC49500A003E432C4D41432C253032C1
:10157C0062583A25303262583A25303262583A2550
:10158C00303262583A25303262583A25303262583D
:10159C002C4D414320E0E4F0E5F10A003E432C568B
:1015AC0045522C20332E3220EEF220257320257349
:1015BC002CC2E5F0F1E8FF20495020ECEEE4F3EB0F
:1015CC00FF0A004A756E203330203230303800313B
:1015DC00323A30393A3236003E432C4C442C50527D
:1015EC004F473A202020202020202020202020207F
:1015FC0020202020202020202020202020202020DF
:10160C0020202020202020202020202020202020CE
:10161C0020202020202020202020202020202020BE
:10162C0020202020202020202CC4E0F2E020EFF00D
:10163C00EEF8E8E2EAE828F4E0E9EB290A003E2AB1
:10164C002C312CCEF1EDEEE2EDFBE520EFE0F0E0FD
:10165C00ECE5F2F0FB20F1E5F2E5E2EEE3EE20E85A
:10166C00EDF2E5F0F4E5E9F1E00A003E412C413001
:10167C00312C2562752E2562752E2562752E2562FC
:10168C00752C495020E0E4F0E5F120E0E4E0EFF2C5
:10169C00E5F0E00A003E412C4130322C2562752EDB
:1016AC002562752E2562752E2562752C495020E019
:1016BC00E4F0E5F120EEF1ED2E20F1E5F0E2E5F0BD
:1016CC00E00A003E412C4130332C2562752E2562F8
:1016DC00752E2562752E2562752C495020E0E4F09C
:1016EC00E5F120F0E5E72E20F1E5F0E2E5F0E00A87
:1016FC00003E412C4130342C2562752E2562752E0E
:10170C002562752E2562752CCCE0F1EAE020F1E51E
:10171C00F2E80A003E412C4130352C2562752E250D
:10172C0062752E2562752E2562752CD8EBFEE70AA4
:10173C00003E2A2C312CC4EEEF2E20EFE0F0E0EC32
:10174C00E5F2F0FB20F1E5F2E5E2EEE3EE20E8ED68
:10175C00F2E5F0F4E5E9F1E00A003E422C533031B9
:10176C002C2562752CC6E4E0F2FC20E7E0EFF0EEED
:10177C00F1E020F1EEE5E4E8EDE5EDE8FF20EEF236
:10178C0020F1E5F0E2E5F0E00A003E422C53303265
:10179C002C2562752CCEE1ECE5ED20F120F1E5F085
:1017AC00E2E5F0EEEC20E1E5E720EAE2E8F2E0ED3C
:1017BC00F6E8E90A003E422C5330332C2562752C96
:1017CC00CFE5F0E5E7E0EFF3F1EA20EFF0E820EF0A
:1017DC00EEF2E5F0E520F1E2FFE7E820F120F1E59B
:1017EC00F0E2E5F0EEEC0A003E422C5330352C25AD
:1017FC0062752CCAE0EDE0EB20F8E8F0EEEAEEE2E0
:10180C00E5F8E0F2E5EBFCEDEEE3EE20EEE1ECE5E5
:10181C00EDE00A003E532C5330362C253032625802
:10182C0025303262582530326258253032625825C4
:10183C003032625825303262582C4D414320E0E45E
:10184C00F0E5F120F8E8F0EEEAEEE2E5F8E0F2E59A
:10185C00EBFCEDEEE3EE20EEE1ECE5EDE00A003E14
:10186C00454E440A000A44756D70582020202020F3
:10187C0030302030312030322030332030342030A2
:10188C003520303620303720303820303920304168
:10189C002030422030432030442030452030460A4E
:1018AC00000A3A003A20000A000A44756D70442080
:1018BC002020202030302030312030322030332096
:1018CC00303420303520303620303720303820303E
:1018DC0039203041203042203043203044203045E4
:1018EC0020304600457272206B6579005264206589
:1018FC006570726F6D0A005264204D454D0A00529E
:10190C006420436F64650A00577269746520436FE5
:10191C0064650A0044656275674950204F4E0A00A1
:10192C0044656275674950204F46460A004465621B
:10193C00756755736572204F6E0A00446562756752
:10194C0055736572204F46460A0044656275674DB3
:10195C007367204F6E0A0044656275674D7367208C
:10196C004F46460A00436F6E666967206C6F636B67
:10197C00210A00577220656570726F6D0A00205342
:10198C0061766520656570726F6D210A0045727213
:10199C00204D414321004C6F61643E3E002A003CC7
:1019AC004130313D003C4130323D003C4130333D13
:1019BC00003C4130343D003C4130353D003C210081
:1019CC003C5330313D003C5330323D003C533033BE
:0E19DC003D003C5330353D003C5330363D005D
:063D1000016700016500DF
:104A7F00C28E438910E4F58B758DB8D2ABD28E22DE
:03001B00023FCCD5
:103FCC00C0E0C083C082C0D0C28E758B00758DB826
:103FDC00201C0675A61E75A6E10565D218E567605E
:103FEC00020567E566D3940140021566056AE56A29
:103FFC00540F7048D224E56A543F7012D216906662
:10400C008BE0600A04F0E0D394B44002D21C9066BA
:10401C0086E0600204F0906104E0600214F09066A7
:10402C008CE0D394014003E014F0301B020568E5EA
:10403C0069D394644004D21C80020569E564D3946E
:10404C000140021564D28ED0D0D082D083D0E03221
:100F6300C2AFC2217D027C007F07124A488F45E54C
:100F730045646060097D017F601249E0D221E4FD90
:100F8300FC7F0B124A488F45E54530E6097D04E4B2
:100F9300FF124A04D2217D017C007F07124A488F49
:100FA30045E5457008FD7FFF1249E0D2213021035A
:100FB300126000C288C2A8C2AA758900123F30908D
:100FC30063497403F0A374CCF0E4906348F0123CDB
:100FD30046122CADC21C124698D221C223C22290C3
:100FE30065767408F09062B47424F0E4A3F090631F
:100FF3003EE09062B6F090633FE09062B7F090639A
:1010030040E09062B8F0906341E09062B9F0906381
:1010130042E09062BAF0906343E09062BBF0756681
:1010230001E4906577F0C21DC21EC21FC2202021B9
:1010330018AF45FE7D031239B1E4FF123DD07E1592
:101043007F2CE4FBFDFC1235C790668BE0600374D4
:1010530001F0E4906104F0F568906575F0F56912AC
:101063004A7F75A70775A61E75A6E1D2AFE4F56999
:10107300906104E0700312090E90668CE0B40111D4
:101083009080007410F0E490668CF0D221C222C2EA
:1010930023908008E0F54530E405D21D7410F0E597
:1010A3004530E508D21F9080087420F0E54530E60E
:1010B30008D21E9080087440F0E568C39403401979
:1010C300908002E4F0908001F0908000F0E5689455
:1010D300064006E4F5681246989080A0E07003127B
:1010E30044869080B8E070031245009080D0E07091
:1010F3000312457A908000E07013301D101236CE33
:10110300906331EFF0D394004003120036908002D5
:10111300E07006908000E06005D21B021070C21BD5
:10112300E4F568906104E0600302107020211290DE
:101133006578E0600C7E157F2E1238C9E4906578DF
:10114300F0301F1212331C906331EFF0D394004040
:1011530005E0FF120032201E030212D41230189051
:101163006331EFF07003021070906375E054BF2495
:101173007F700302123D14700302121524026003F0
:101183000212762021077E157F351238C9202503E8
:101193000212D490634DE0FF7006906351E06061EA
:1011A300906682E0FEB50722A3E0FF90634EE0B5B0
:1011B3000718906684E0FF90634FE0B5070C9066D4
:1011C30085E0FF906350E06F6037906351E06E609D
:1011D300030212D4906683E0FF906352E06F6003D2
:1011E3000212D4906684E0FF906353E06F600302C1
:1011F30012D4906685E0FF906354E06F600302129F
:10120300D4C2199065777401F0124AE2756601023F
:1012130012D490668BE060037401F090667AE0FF6D
:10122300906377E06F60030212D490667AE004F073
:10123300E4F566906575F00212D43019030212D4F6
:10124300906344E07003021070906355740AF012C7
:10125300481FD219E4F566906575F090668604F030
:10126300E4906679F0A3F02021677E157F4312385E
:10127300C9805E90668BE060037401F03019529070
:101283006375E020E74B906377E0FF906679E0FEBB
:101293006F600D906681E07007EE146F70338013FA
:1012A300906679E004F0906331E0FFD39404400347
:1012B300123E809060007482F0A37401F090637713
:1012C300E0906002F07E607F007D0312416F0210A8
:1012D300702019030213ECE566706812485BEF6037
:1012E300237E647F75906476E02404FD12416F9041
:1012F3006681E07009906355E0F566021070E4F5CD
:1013030066021070906686E0D3943C403690668106
:10131300E0703090668604F0123B6DE4906475F0E3
:10132300A37412F090667AE0906477F0A374FDF0F2
:1013330090610563A20190647963A2017F12122B6D
:101343009F809E124AD08F45E545B40115906000F9
:101353007483F0E4A3F07E607F007D0212416F028C
:101363001070E545D39401401C9060007483F0A392
:101373007401F0E54524FEA3F07E607F007D031237
:10138300416F021070E5666401600302107090659E
:1013930075E004F02021077E157F4D1238C9906354
:1013A30055E0C394C85004E02432F0906575E0C35F
:1013B3009405400DC219E4906577F0124AE20210D9
:1013C300707C667D82906349E0FAA3E0FB7F0212A2
:1013D30043007E647F75906476E02404FD12416FC0
:1013E300906355E0F566021070E5666401600302E0
:1013F3001070906577E014604624FE604214700319
:101403000214DF24046003021070E4F5682025133E
:101413009065777404F0906575E05401F07566018A
:101423000210709080027410F0E4906577F090657C
:101433007504F07566FA90668274FFF0021070907E
:101443006682E070030214C99064757480F090643E
:10145300777401F0E4A3F0A304F0A37430F0A37451
:101463007BF0E4F545747C2545F582E43464F5832B
:10147300747DF0747D2545F582E43464F583E4F0EE
:10148300E5452407906476F07C667D82906349E0AD
:10149300FAA3E0FB7F021243007E647F75E54524D7
:1014A30009FD12416F906681E0601B12481FD2193B
:1014B300E4F566906575F090668604F0E4906679CD
:1014C300F0A3F0021070302507E4906577F08006F2
:1014D3009065777404F07566FA0210709080027458
:1014E30010F0756605906575E06401FFF09065770F
:1014F3007401F0EF7019906351E06013FCA3E0FDF9
:10150300A3E0FEA3E0FF9066821227790210709099
:10151300634DE0FCA3E0FDA3E0FEA3E0FF90668241
:0815230012277902107080FE0E
:01152B00229D
:10003600906376E0B444047F0180027F009063758C
:10004600E0B447047E0180027E00EE5F604A906362
:100056003EE0906377F090633FE0906378F09063C2
:1000660040E0906379F0906341E090637AF09063AA
:1000760042E090637BF0906343E090637CF0906392
:10008600767452F09062AE63A2019080A863A201DA
:100096007F06122B9F020904906331E0C394085037
:1000A6000302090D90633EE0FF906377E06F600303
:1000B60002090D90633FE0FF906378E06F600302F2
:1000C600090D906340E0FF906379E06F60030209D9
:1000D6000D906341E0FF90637AE06F600302090DC3
:1000E600906342E0FF90637BE06F600302090D902E
:1000F6006343E0FF90637CE06F600302090D906349
:1001060076E0B444159062AEE0B4FF0E63A20190AF
:1001160080A863A2017F06122B9F90668BE0600386
:100126007401F090668C7464F09063767452F0906B
:100136006375E0646D60030202957BFF7A1579585A
:100146001222E57BFF7A15797290633EE0F54EA3A5
:10015600E0F54FA3E0F550A3E0F551A3E0F552A377
:10016600E0F5531222E5754EFF754F157550CF75A4
:1001760051FF7552157553DB7BFF7A1579A812224C
:10018600E57BFF7A1579E41222E57BFF7A16794A38
:100196001222E57BFF7A167977906344E0F54EA349
:1001A600E0F54FA3E0F550A3E0F5511222E57BFF01
:1001B6007A1679A190634DE0F54EA3E0F54FA3E0E2
:1001C600F550A3E0F5511222E57BFF7A1679CF9020
:1001D6006351E0F54EA3E0F54FA3E0F550A3E0F53B
:1001E600511222E57BFF7A1679FD90633AE0F54ECF
:1001F600A3E0F54FA3E0F550A3E0F5511222E57B0D
:10020600FF7A177920906336E0F54EA3E0F54FA309
:10021600E0F550A3E0F5511222E57BFF7A17793D10
:100226001222E57BFF7A177966A225E433F54E1292
:1002360022E57BFF7A177996906681E0F54E1222C9
:10024600E57BFF7A1779C190668BE0F54E1222E5C1
:100256007BFF7A1779F4A217E433F54E1222E57B79
:10026600FF7A18792090667BE0F54EA3E0F54FA360
:10027600E0F550A3E0F551A3E0F552A3E0F55312E3
:1002860022E51234827BFF7A18796B1222E52290DE
:100296006375E0644C60030203547E187F71FBFDB6
:1002A600FC1235C790637DE0F546A3E0F547E4F51B
:1002B60049E4F548854782854683E0FF747F2548F3
:1002C600F582E43463F583EFF00548E548B410E4BD
:1002D600E54690637FF0A3E547F07E187FAD7C632B
:1002E6007D7F7B021235C7E4F548854782854683C4
:1002F600E0FF747F2548F582E43463F583EFF0056B
:1003060047E547700205460548E548B410DC7E1807
:100316007FB07C637D7F7B101235C7E4F548854747
:1003260082854683E0FF747F2548F582E43463F5D1
:1003360083EFF00548E548B410E40549E549C39460
:100346001050030202B77E187FB31238C922906399
:1003560075E0646C60030203F5F54A7E187FB5FB11
:10036600FDFC1235C7E4F549E4F548A84AE6FF74F2
:100376007F2548F582E43463F583EFF00548E548C8
:10038600B410E8E490637FF0A3E54AF07E187FADF1
:100396007C637D7F7B021235C7E4F548A84AE6FFF9
:1003A600747F2548F582E43463F583EFF0054A054A
:1003B60048E548B410E67E187FB07C637D7F7B10ED
:1003C6001235C7E4F548A84AE6FF747F2548F5824A
:1003D600E43463F583EFF00548E548B410E80549D1
:1003E600E549C3940840817E187FB31238C922902C
:1003F6006375E0644B7061F54874672548F582E4DF
:100406003463F583E0603274672548F582E434632B
:10041600F583E0F4602374672548F582E43463F5D8
:1004260083E0FF747D2548F582E43463F583E0B507
:1004360007100548E548B408C09061047432F0021C
:1004460009049063757421F03021030209047E18B3
:100456007FF01238C9020904906375E0B4521A207D
:1004660021077E187FF81238C99063757472F07E82
:10047600637F757D081240E822906375E0644970D9
:10048600452021077E197F031238C990637DE0F568
:1004960046A3E0F547E4F548854782854683E0FFB5
:1004A600747F2548F582E43463F583EFF00547E56C
:1004B60047700205460548E548B480DC7E637F75D3
:1004C6007D8A1240E822906375E0644370462021DD
:1004D600077E197F0B1238C990637DE0F546A3E0CD
:1004E600F547E4F548854782854683E493FF747FA4
:1004F6002548F582E43463F583EFF00547E5477058
:100506000205460548E548B480DB7E637F757D8A33
:100516001240E822906375E0645A70532021077EEA
:10052600197F141238C990637DE0F546A3E0F547BC
:100536007C637D7F7B80AF47AE46124906E4F54873
:10054600854782854683E493FF747F2548F582E4D8
:100556003463F583EFF00547E54770020546054825
:10056600E548B480DB7E637F757D8A1240E8229081
:100576006375E06444600302060690637DE0FF64F1
:10058600447003020904EFB4310CC2217E197F20A6
:100596001238C902090490637DE0B4300CD2217E82
:1005A600197F2C1238C902090490637DE0B4320C1D
:1005B600D2227E197F391238C902090490637DE080
:1005C600B4330CC2227E197F471238C9020904903F
:1005D600637DE0B4340CD2237E197F561238C902EB
:1005E600090490637DE0B4350CC2237E197F631243
:1005F60038C902090490637DE0FF12001E02090457
:10060600906104E070132021077E197F711238C9AA
:100616009063757421F00209049061047432F090BD
:100626006375E0FFB45104C2AF80FEEF64577045B6
:100636002021077E197F7F1238C990637EE0906380
:1006460031F0E4F548906331E0FFE548C39F40038D
:10065600020904747F2548F582E43463F583E0FFDC
:1006660090637DE0254824ADF582E43461F583EF9F
:10067600F0054880D0906375E06453600302072854
:100686002021077E197F8A1238C990633EE0FF90C9
:1006960061B6E06F703C90633FE0FF9061B7E06F3A
:1006A6007030906340E0FF9061B8E0B50724906336
:1006B60041E0FF9061B9E0B50718906342E0FF9012
:1006C60061BAE0B5070C906343E0FF9061BBE06F51
:1006D60060169063757421F03021030209047E19B7
:1006E6007F991238C9020904E4F548E4F56974AD46
:1006F6002548F582E43461F583E0FDAF481249668A
:100706000548E548C394FE40E2C2AFE4907FF0F0AE
:10071600A3F0907FFD74AAF0A374FFF0A37455F0C4
:1007260080FE906375E0644F704C90637DE0F54603
:10073600A3E0F547E5474546700A2021077E197F65
:10074600A21238C92021077E197FA91238C9E4F5FB
:1007560048747F2548F582E43463F583E085478253
:10076600854683F00547E547700205460548E54896
:10077600B480DE020904906375E0FFB445219063FE
:100786007DE0FDA3E0907FF0CDF0A3EDF0C2AF9049
:100796007FFD74AAF0A374FFF0A37455F080FEEFFA
:1007A6006465600302090D90637DE0FFA3E0907F1E
:1007B600F0CFF0A3EFF0E4F546F547D3907FF1E0F4
:1007C6009547907FF0E095464021E4F5692547FF7F
:1007D600E5463478FE7B80AD47AC46124906748008
:1007E6002547F547E43546F54680D07E197FAB129E
:1007F60041F6EF4E6020120003906344EFF01200C2
:1008060003906345EFF0120003906346EFF0120089
:1008160003906347EFF07E197FB11241F6EF4E6009
:100826002012000390634DEFF012000390634EEF29
:10083600F012000390634FEFF0120003906350EF45
:10084600F07E197FB71241F6EF4E6020120003903A
:100856006351EFF0120003906352EFF01200039021
:100866006353EFF0120003906354EFF07E197FBDDF
:100876001241F6EF4E602012000390633AEFF01239
:10088600000390633BEFF012000390633CEFF0121D
:10089600000390633DEFF07E197FC31241F6EF4EE1
:1008A6006020120003906336EFF012000390633766
:1008B600EFF0120003906338EFF0120003906339F3
:1008C600EFF0E4F548E4F569E54804FF7436254899
:1008D600F582E43463F583E0FD1249660548E54890
:1008E600C3944340E0C2AFE4907FF0F0A3F0907F62
:1008F600FD74AAF0A374FFF0A37455F080FE7E6326
:070906007F757D081240E837
:01090D0022C7
:1048CE00AE07EEC39430400BEED394395005EE2470
:1048DE00D0FF22EEC39461400BEED394665005EEEA
:1048EE0024A9FF22EEC39441400BEED3944650050B
:0848FE00EE24C9FF22AF0622DF
:104A65009062ADE004F070069062ACE004F09062F4
:0A4A7500ACE0FEA3E0FF1247DD22D3
:10000300124A651248CEEFC454F0FEC006124A6588
:080013001248CED0E02FFF22BD
:10463B00E4906B25F0124A65906B26EFF0C3943033
:10464B004018E0FFD394395011906B25E02405F509
:10465B0082E43461F583EFF08011906B25E0240543
:10466B00F582E43461F583E4F0800C906B25E00473
:10467B00F0E0D3940840BE75540075550075560094
:0C468B00E4F5577B017A617905122E746A
:014697002200
:0441F6008E4B8F4C11
:1041FA009062ACE4F0A374FFF0124A65EF606EF4CB
:10420A00606B854C82854B83E493B507EC754D0151
:10421A00E54C254DF582E4354BF583E49360259012
:10422A0062ADE0254DFF9062ACE03400FE1247DD3E
:10423A00E54C254DF582E4354BF583E493B5070447
:10424A00054D80CCE54C254DF582E4354BF583E4EC
:10425A009370A6E54D24FFFFE434FFFE9062ADE0C3
:10426A002FF09062ACE03EF07E007F0122E4FEFF78
:01427A002221
:103C46007E197FC91241F6EF4E70037F01227E195D
:103C56007FCC1241F6EF4E600C124A65EF24D02459
:103C6600FF92258002D2257E197FD21241F6EF4EB1
:103C7600600C124A65EF24D0906681F08005E490CE
:103C86006681F07E197FD81241F6EF4E600C124A1B
:103C960065EF24D090668BF08005E490668BF07E0D
:103CA600197FDE1241F6EF4E600C124A65EF24D002
:103CB60024FF92178002C21790633E63A2019066AA
:103CC6007B63A2017F06122B9F30173B7E197FE490
:103CD6001241F6EF4E603012000390667BEFF01251
:103CE600000390667CEFF012000390667DEFF01201
:103CF600000390667EEFF012000390667FEFF012ED
:0A3D06000003906680EFF07F0022BA
:10479600906576E0C3947C503D906576E0FE04F02B
:1047A60074B42EF582E43462F583EFF0BF0A2790E5
:1047B6006576E0FF04F074B42FF582E43462F58385
:1047C600E4F0906576E0FF12427B9065767408F01F
:0747D6009062B5E004F0223F
:104698009080007480F090633663A201F583F58200
:1046A80063A2017F08122B9F90633E63A201908052
:1046B8008863A2017F0A122B9F908092E4F0A37472
:1046C80032F0A37401F0906348E0FF9080B1F0905D
:1046D80080E1EFF09080957455F0A3F0908000741D
:0946E80001F090800974F0F02249
:10448600908009E04410F09080A0E0706C9080A1CC
:104496007482F09080A874FFF0A3F0A3F0A3F07FDD
:1044A600039080AEEFF07FCBA3EFF07F039080AC5C
:1044B600EFF0A374CBF09080007402F0906B1412AE
:1044C600278500000000906B14E0908040F0906B10
:1044D60015E0908041F0906B16E0908042F0906B72
:1044E60017E0908043F0A3E4F0A3F0A3F0A3F090CC
:0944F6008018F0A3F0A3F0A3F07C
:0144FF00229A
:10457A00908009E04440F09080D17482F0906349C1
:10458A00E0FF9080DEF090634AE0FF9080DFF090D9
:10459A0080027402F0906B181227850000000090C8
:1045AA006B18E0908058F0906B19E0908059F09069
:1045BA006B1AE090805AF0906B1BE090805BF0A33E
:1045CA00E4F0A3F0A3F0A3F0908030F0A3F0A3F0FE
:0245DA00A3F04C
:0145DC0022BC
:10450000908009E04420F09080B8E0706C9080B911
:104510007482F07F039080C6EFF07FCDA3EFF07F31
:10452000039080C4EFF0A374CDF09080C074FFF0CE
:10453000A3F0A3F0A3F09080017402F0906B1C1222
:10454000278500000000906B1CE090804CF0906B81
:104550001DE090804DF0906B1EE090804EF0906BCF
:104560001FE090804FF0A3E4F0A3F0A3F0A3F0903D
:094570008024F0A3F0A3F0A3F0F5
:01457900221F
:104300008C468D47A907EAFDE975F018A424ACFF97
:10431000E5F034808F82F583EDF0EBFDE975F01860
:10432000A4FFAEF024ACFBEE34808B82F583A3EDCA
:10433000F08547828C83E0FDEF24A8FFEE3480FEF9
:104340008F82F583EDF08547828C83A3E08F828E88
:1043500083A3F0854782854683A3A3E0FDE975F03A
:1043600018A424A8FFE5F03480FE8F82F583A3A370
:10437000EDF08547828C83A3A3A3E08F828E83A375
:04438000A3A3F022E1
:0640E8008D4BAB07AA0698
:1040EE00908000E030E5079065787401F022906BC7
:1040FE0014E0FCA3E0FDA3E0FEA3E0F54F8E4E8D91
:10410E004D8C4CAE02AF038E838F8263A201E54EBF
:10411E00540744C0F583854F8263A201AF4B122C26
:10412E0011E4FCFDFEE54F254BF54FEE354EF54EF9
:10413E00ED354DF54DEC354CF54C908040E54CF0A1
:10414E00A3E54DF0A3E54EF0A3E54FF0908000748B
:10415E0020F0AF4FAE4EAD4DAC4C906B1412277994
:01416E00222E
:06416F008D46AB07AA0615
:10417500908002E030E5079065787403F022906B3B
:1041850018E0FCA3E0FDA3E0FEA3E0F54A8E498D0F
:10419500488C47AE02AF038E838F8263A201E54947
:1041A500540744D0F583854A8263A201AF46122C99
:1041B50011E4FCFDFEE54A2546F54AEE3549F5498B
:1041C500ED3548F548EC3547F547908058E547F01B
:1041D500A3E548F0A3E549F0A3E54AF09080027411
:1041E50020F0AF4AAE49AD48AC47906B181227791D
:0141F50022A7
:023DD0008F461C
:103DD200908001E030E5099065787402F07F00225E
:103DE200906B1CE0FCA3E0FDA3E0FEA3E0F54A8E8D
:103DF200498D488C4790667B63A201E5495407448C
:103E0200C8F583854A8263A2017F06122C27E54A00
:103E12002406F54AE43549F549E43548F548E435E0
:103E220047F54790657963A201E549540744C8F50F
:103E320083854A8263A201AF46122C27E4FCFDFE71
:103E4200E54A2546F54AEE3549F549ED3548F54846
:103E5200EC3547F54790804CE547F0A3E548F0A3E1
:103E6200E549F0A3E54AF09080017420F0AF4AAE34
:0D3E720049AD48AC47906B1C122779AF4654
:013E7F002220
:1036CE009081E0E0F5460546054605460546054669
:1036DE0005460546054605460546908010E0F54927
:1036EE00A3E0F54AA3E0F54BA3E0F54C9081E1E0B1
:1036FE00F546054605460546054605460546054674
:10370E00054605460546908014E0F54DA3E0F54EBE
:10371E00A3E0F54FA3E0F550E54FB54B08E550B5E6
:10372E004C037F0022E4F546E54F540744E0F58351
:10373E0085508263A20190637563A2017F08122CEB
:10374E005790637763A2019062AE63A2017F061267
:10375E002B9F906375E0F547A3E0F548E4F546909E
:10376E006375E0702AA3E024F8F546E54F5407444C
:10377E00E0F58385508274082582F582E43583F561
:10378E008363A20190637563A201AF46122C57AEFC
:10379E0047E4FCFDE5502548F550E54F3EF54FED6D
:1037AE00354EF54EEC354DF54D908014E54DF0A3AC
:1037BE00E54EF0A3E54FF0A3E550F0908000744085
:0337CE00F0AF4613
:0137D10022D5
:103018009081E6E0F546054605460546054605461F
:1030280005460546054605460546908028E0F549CB
:10303800A3E0F54AA3E0F54BA3E0F54C9081E7E067
:10304800F546054605460546054605460546054630
:1030580005460546054690802CE0F54DA3E0F54E63
:10306800A3E0F54FA3E0F550E4F546E54FB54B0A6C
:10307800E550B54C05C21E023184E54F540744F0B3
:10308800F58385508263A20190637563A2017F086E
:10309800122C57906375E0F547A3E0F548E54845DD
:1030A8004770099080027410F07F0022906682E0D9
:1030B800FFF46030906377E06F600302314B9066F5
:1030C80083E0FF906378E06F7079906684E0FF900A
:1030D8006379E06F706D906685E0FF90637AE06FCA
:1030E8006031805F906377E0906682F0906378E06B
:1030F800906683F0906379E0906684F090637AE05C
:10310800906685F090637BE0FFA3E0906349CFF081
:10311800A3EFF0906375E0702AA3E024F8F546E584
:103128004F540744F0F58385508274082582F58250
:10313800E43583F58363A20190637563A201AF460A
:10314800122C57AE47E4FCFDE5502548F550E54FF5
:103158003EF54FED354EF54EEC354DF54DAF4CAED9
:103168004BAD4AAC49AB50AA4FA94EA84DD3122734
:103178006840099080027410F07F002290802CE54E
:103188004DF0A3E54EF0A3E54FF0A3E550F0908095
:06319800027440F0AF4696
:01319E00220E
:10331C009081E3E0F546054605460546054605461B
:10332C000546054605460546054690801CE0F549D0
:10333C00A3E0F54AA3E0F54BA3E0F54C9081E4E063
:10334C00F546054605460546054605460546054629
:10335C00054605460546908020E0F54DA3E0F54E68
:10336C00A3E0F54FA3E0F550E4F546E54FB54B0A65
:10337C00E550B54C05C21F023467E54F540744E8CD
:10338C00F58385508263A20190600463A2017F0ED5
:10339C00122C6D906004E0F547A3E0F54890600CAA
:1033AC00E0FFF4604590667BE0FEEF6E706EA3E08C
:1033BC00FF90600DE06F706490667DE0FF90600E92
:1033CC00E06F705890667EE0FF90600FE06F704C7D
:1033DC0090667FE0FF906010E06F7040906680E038
:1033EC00FF906011E06F60048032D2D9906004E0ED
:1033FC00702AA3E024F2F546E54F540744E8F58320
:10340C00855082740E2582F582E43583F58363A2A0
:10341C000190600463A201AF46122C6DAE47E4FC30
:10342C00FDE5502548F550E54F3EF54FED354EF591
:10343C004EEC354DF54DAF4CAE4BAD4AAC49AB50A7
:10344C00AA4FA94EA84DD31227685006E548454708
:10345C0070099080017410F07F0022908020E54D5F
:10346C00F0A3E54EF0A3E54FF0A3E550F0908001FA
:05347C007440F0AF46B2
:013481002228
:0438C9008E4B8F4C47
:1038CD00908000E030E5079065787401F022906BF0
:1038DD0014E0FCA3E0FDA3E0FEA3E0F5528E518DB4
:1038ED00508C4FE552FFE5515407FEE42FF54EEE97
:1038FD0034C0F54D854E82F5837423F0054EE54EAB
:10390D007002054D534DC7F582854D83740AF00540
:10391D004EE54E7002054D534DC790633E63A201B7
:10392D00854D83854E8263A2017F06122C1174068C
:10393D00254EF54EE4354DF54D854B83854C826313
:10394D00A201854D83854E8263A201122BF5E4FC05
:10395D00FDFE906B14E0F8A3E0F9A3E0FAA3E02FCD
:10396D00FFEE3AFEED39FDEC38FCEF2408FFE43EA6
:10397D00FEE43DFDE43CFC906B14122779906B1432
:10398D00E0908040F0906B15E0908041F0906B16C8
:10399D00E0908042F0906B17E0908043F0908000B3
:0339AD007420F093
:0139B00022F4
:0A35C7008E4D8F4E8C4F8D508B51AE
:1035D100908000E030E5079065787401F022906BEF
:1035E10014E0FCA3E0FDA3E0FEA3E0F5578E568DA9
:1035F100558C54E557FFE5565407FEE42FF553EE7D
:1036010034C0F552855382F5837423F00553E55395
:10361100700205525352C7F582855283740AF00530
:1036210053E553700205525352C790633E63A201A2
:1036310085528385538263A2017F06122C11740681
:103641002553F553E43552F552854D83854E8263FA
:10365100A20185528385538263A201122BF58F58F3
:10366100EF2553F553E43552F552E5516017854F77
:103671008385508263A20185528385538263A201AF
:10368100AF51122C11E55824082551F551FFE4FCE6
:10369100FDFEE5572FF557EE3556F556ED3555F547
:1036A10055EC3554F554908040E554F0A3E555F0C0
:1036B100A3E556F0A3E557F09080007420F0AF57D2
:0C36C100AE56AD55AC54906B1412277936
:0136CD0022DA
:063A92008E478F488D49AC
:103A9800908000E030E5079065787401F022906B23
:103AA80014E0FCA3E0FDA3E0FEA3E0F54F8E4E8DED
:103AB8004D8C4CE54FFFE54E5407FEE42FF54BEED9
:103AC80034C0F54A854B82F5837423F0054BE54BEA
:103AD8007002054A534AC7F582854A83EBF0054BC5
:103AE800E54B7002054A534AC790633E63A20185BD
:103AF8004A83854B8263A2017F06122C1174062526
:103B08004BF54BE4354AF54A85478385488263A2DD
:103B180001854A83854B8263A201AF49122C117437
:103B2800082549F549FFE4FCFDFEE54F2FF54FEE6A
:103B3800354EF54EED354DF54DEC354CF54C908048
:103B480040E54CF0A3E54DF0A3E54EF0A3E54FF0BA
:103B58009080007420F0AF4FAE4EAD4DAC4C906BE2
:043B68001412277993
:013B6C002236
:02427B008F5F53
:10427D00908000E030E5079065787401F022906B36
:10428D0014E0FCA3E0FDA3E0FEA3E0F5638E628DD8
:10429D00618C60E563FFE5625407FEE42FFFEE34A9
:1042AD00C09062B463A201F5838F8263A201AF5FF8
:1042BD00122C11E4FCFDFEE563255FF563EE35621E
:1042CD00F562ED3561F561EC3560F560908040E5A6
:1042DD0060F0A3E561F0A3E562F0A3E563F09080E3
:1042ED00007420F0AF63AE62AD61AC60906B1412E0
:0242FD0027791F
:0142FF00229C
:0639B1008E468F47AB05B6
:1039B700908000E030E5079065787401F022906B05
:1039C70014E0FCA3E0FDA3E0FEA3E0F54D8E4C8DD3
:1039D7004B8C4AE54DFFE54C5407FEE42FF549EEC5
:1039E70034C0F548854982F5837423F00549E549D4
:1039F700700205485348C7F582854883EBF00549AF
:103A0700E5497002054890633E63A20185488385B6
:103A1700498263A2017F06122C1174062549F549D4
:103A2700E43548F5485348C7E546854982854883C4
:103A3700F00549E549700205485348C7F5828548AE
:103A470083E547F00549E549700205485348C7E54E
:103A57004D240AF54DE4354CF54CE4354BF54BE474
:103A6700354AF54A908040E54AF0A3E54BF0A3E5D7
:103A77004CF0A3E54DF09080007420F0AF4DAE4CB4
:0A3A8700AD4BAC4A906B1412277986
:013A91002212
:0A4AC500E4FEEEC39F50030E80F8DC
:014ACF0022C4
:103F3000E4F546E5462401FFE433FE1247DD74361E
:103F40002546F582E43463F583EFF00546E546C384
:103F5000943F40DFE4F546E546247FFFE433FE125C
:103F600047DD742D2546F582E43461F583EFF07466
:103F70002D2546F582E43461F583E0FF6003B4FF4C
:103F80001D742D2546F582E43461F5837420F074A8
:103F90002E2546F582E43461F583E4F08009054678
:103FA000E546C3948040B0E49061ACF0F546AF467E
:103FB0007E001247DD74AD2546F582E43461F58359
:0B3FC000EFF00546E546C394FE40E329
:013FCB0022D3
:104A2800E4FDFCC3ED9FEC9E5015E4FBFA0BBB00C4
:0F4A3800010ABA01F8BB90F50DBD00010C80E436
:014A4700224C
:0D4A9E004390014390025390FE5390FD227F
:0D4AAB005390FD5390FE4390024390012272
:0E4A8F005390FD439002E5905408FF5390FDB4
:014A9D0022F6
:0D4AB8005390FD4390014390025390FD2266
:074ADB00AE071FEE70FA2286
:02493A00AD07C7
:10493C00E4FC5390FDEDA804088002C333D8FC308E
:10494C00E70543900180035390FE7F05124ADB4339
:09495C0090020CBC08DC5390FD34
:01496500222F
:10499000E4FF5390FD7E07439002E59030E00D74F4
:1049A00001A806088002C333D8FC42075390FD1EBD
:0849B000C3EE6480948050DF27
:0149B80022DC
:10496600AB05AA07124A9E7FA012493A124A8FAF98
:104976000212493A124A8FAF0312493A124A8F126B
:0A4986004AAB7F0A7E00124A282285
:0447DD00AB07AA0676
:1047E100C3EB94FFEA9400400DE42BF58274773A11
:1047F100F583E493FF22124A9E7FA012493A124A9E
:104801008FAF0312493A124A8F124A9E7FA1124971
:0D4811003A124A8F124990124AB8124AAB6F
:01481E002277
:024906008B4BD9
:10490800A2AF9226C2AF85A24C53A2FE8E838F829D
:1049180005A28C838D827409122C9BE54B53A2FE51
:1049280043A220122C9D53A2DF854CA2A22692AF4F
:01493800FF7F
:01493900225B
:104A4800A2AF9226C2AF8C838D82EF122C9B43A219
:0C4A580020122C9D53A2DFA22692AFFF7B
:014A6400222F
:0249E0008F4600
:1049E200A2AF9226C2AFE4F5838D827406122C9B8D
:1049F200E54643A220122C9D53A2DFA22692AF7F4E
:014A020001B2
:014A03002290
:024A04008F46DB
:104A0600A2AF9226C2AFE4F5838D82740A122C9B64
:104A1600E54643A220122C9D53A2DFA22692AF7F29
:014A2600018E
:014A2700226C
:102AC400A907E7FFA805EF93C3966008403B74FC91
:102AD4002FFF80F00F08EF93C3966008402B74FB20
:102AE4002FFF80E00F08EF93C3966008401B74FA31
:102AF4002FFF80D00F08EF93D3966008400B74F932
:102B04002FFF80C01F1F1F1F1FEF54FEF80303F782
:102B1400E893FC08E893FD08E893FE08E893FF2295
:102B240009E993C39D6008402974FB29F980F109E0
:102B3400E993C39E6008401A74FA29F980E209E90E
:102B440093D39F6008400B74F929F980D31919199C
:102B54001919E9C313C313FF22740093F8ECC39843
:102B64004024701F740193F8EDC3984019701474D5
:0E2B74000293F8EEC398400E7009740393F8B4
:102B8200EFC39840037F00227F0122EDF8E6F008B0
:102B9200A3DFFA22EDF8E0F608A3DFFA22E0A3634E
:102BA200A201F0A363A201DFF475A2002263A201D5
:102BB200F0A363A20122E0A363A201F0A363A20136
:102BC200E0A363A201F0A363A201E463A201F0A364
:102BD20063A201DFE175A20022E0A363A2016DFE00
:102BE200936CFDEE058393FC158363A201DFEA7506
:102BF200A200227F00E493A363A201F00F600CA362
:102C0200E583C2E3F58363A20180EA75A20022E0B4
:102C1200A363A201F0A3E583C2E3F58363A201DF0C
:102C2200EE75A20022E0A363A201F0A3E583C2E451
:102C3200D2E3F58363A201DFEC75A20022E0A36375
:102C4200A201F0A3E58344F8C2E5F58363A201DFA4
:102C5200EC75A20022E583C2E3F583E0A363A2013F
:102C6200F0A363A201DFEE75A20022E583C2E4D2E3
:0A2C7200E3F583E0A363A201F0A3E1
:102C7C0063A201DFEC75A20022E58344F8F583E042
:102C8C00A363A201F0A363A201DFEE75A20022F9F7
:102C9C0022C002C004C00612FFF0D006D004D0023D
:012CAC002205
:10001E00BF360BD209E4F526F527F542F543BF3777
:04002E0002C20922DF
:1045DD00C2A9438902906B0FE0FFF58C8F8A75D9C4
:1045ED000475DA4875DB3175DC4975DD4975DE31E9
:1045FD00E4F5E9F5F9F5EBF5FB906B0DE06016755B
:10460D00EC1075ED10E4F5FCF5FD753E08753C10EC
:10461D00753D01801375EC8075ED80E4F5FCF5FDBD
:0E462D00753E80F53C753D10E4F5EEF5FE227D
:10489500E4FEAF8CEFFD906B0EE07003A3E06D605E
:1048A500051245DD7E01E5D920E2057E021245DDD2
:1048B500E58920E1051245DD7E03D28C75D840756A
:0848C500B740D2AED2AFAF063E
:0148CD0022C8
:0300330002319FF8
:0B319F00C0E0C083C082C0D075D00823
:1031AA00C2AF30DC56C3E5EC95EEC3953E5012E54E
:1031BA003D25ECF5EC30D70405FC801685FCFC8037
:1031CA0011C3E5EC953DF5EC30D70415FC80038579
:1031DA00FCFC300924852782852683E590F00527A3
:1031EA00E52770020526F582852683E5EEF0052798
:1031FA00E5277002052653260FC2DC30D92930098B
:10320A0024852782852683E590F00527E527700225
:10321A000526F582852683E5EBF00527E52770026A
:10322A00052653260FC2D930DA69E53C700405FC3D
:10323A008010E53C25ECF5EC30D70405FC800385CD
:10324A00FCFC300A4CE5285480FFE52825E0F528E7
:10325A003097020528200803632801302F19E52832
:10326A0054E06544702BEF7028753F08F53A8528BD
:10327A002BF528C22F801A053FE53F5407701253D9
:10328A003F3FE53F131313541F242AF8A628752835
:10329A0000C2DA30DB71E53C700405FD8010E53CC4
:1032AA0025EDF5ED30D70405FD800385FDFDE540EC
:1032BA00653B6029E53B54077013E53B1313135430
:1032CA001F2432F8E6F5292007036329FFE529338D
:1032DA009296E52925E0F529053B533B3FB292300A
:1032EA000923852782852683E590F00527E527703F
:1032FA00020526F582852683E4F00527E527700274
:09330A00052653260FC2DBD2AFE9
:09331300D0D0D082D083D0E0328A
:101E6F004241554400575F4D4F44454D00494E5632
:101E7F005F52454300494E565F5452414E530049FD
:101E8F004E565F414C4C004C495354454E004E5FEB
:101E9F004B50005052494F520047525F5449540023
:101EAF00575F414E535700003E2A2C312CCFE0F0A4
:101EBF00E0ECE5F2F0FB20F1E8EDF5F0EEEDEDEE04
:101ECF00E3EE20EFEEF0F2E00A003E4C2C42303110
:101EDF002C256C752CD1EAEEF0EEF1F2FC20EEE140
:101EEF00ECE5EDE02C35302C3130302C3230302C0D
:101EFF003330302C3630302C313230302C323430CD
:101F0F00302C343830300A003E422C4731302C25EB
:101F1F0062752CC8EDE2E5F0F1E8FF20EDE020EF6F
:101F2F00F0E8B8ECE50A003E422C4731312C25622F
:101F3F00752CC8EDE2E5F0F1E8FF20EDE020EFE5CC
:101F4F00F0E5E4E0F7E50A003E422C4730322C255D
:101F5F0062752CD3EFF0E0E2EBE5EDE8E520EFEE74
:101F6F00F2EEEAEEEC2020285254532D435453291D
:101F7F000A003E532C4730332C256C752CC7E0E4F8
:101F8F00E5F0E6EAE020F1F2E0F0F2E020EFE5F034
:101F9F00E5E4E0F7E828ECF1290A003E532C47303E
:101FAF00332C256C752C202AE7E0E4E5F0E6EAE017
:101FBF0020F1F2E0F0F2E020EFE5F0E5E4E0F7E801
:101FCF0028ECF1290A003E532C4732302C256C7532
:101FDF002CC2F0E5ECFF20EEE6E8E4E0EDE8FF20B0
:101FEF00EEF2E2E5F2E028ECF1290A003E2A2C316C
:101FFF002CC0E4E0EFF2E5F020F1E8EDF5F0EEEDC6
:10200F00EDEEE3EE20EAE0EDE0EBE02E20CFF0EE98
:10201F00F2EEEAEEEB20D2CC3132300A003E422C07
:10202F004B30342C2562752CD0E5E6E8EC20EFF030
:10203F00EEF1EBF3F8EAE820EAE0EDE0EBE020F177
:10204F00E2FFE7E80A003E532C4B30312C25732C6E
:10205F00D1EFE8F1EEEA20CACF0A003E532C4B3005
:10206F00322C25732CCAEEEB2DE2EE20E3F0F3EFCA
:10207F00EF20D2C8D20A003E532C4B30332C25739D
:10208F002CCFF0E8EEF0E8F2E5F220CED220EA20F5
:10209F00C7C3D2C8D20A003C21003C4230313D00B8
:1020AF003C4731303D003C4731313D003C473032F9
:1020BF003D003C4730333D003C4732303D003C4B08
:1020CF0030343D003C4B30313D003C4B30323D0015
:1020DF003C4B30333D000ACFEEEFFBF2EAE020EE4F
:1020EF00F2EFF0E0E2EAE820F1EBE8F8EAEEEC20BC
:1020FF00E4EBE8EDEDEEE3EE20EFE0EAE5F2E021D0
:10210F00000ACEF2EFF0E0E2EAE020D2D30A000AB2
:10211F00CEF2EFF0E0E2EAE020E7E0EFF0EEF1E000
:10212F0020EEF220F1E5F0E2E5F0E00A000A43527A
:10213F0043206572726F72212020000ACFF0E8B839
:10214F00EC20E8EDF4EEF0ECE0F6E8E82020000AF1
:10215F00D7F3E6EEE920CACF212020000AC6E4E03B
:10216F00EB20E8EDF4F320E020F2F3F220F7F2EEAB
:10217F002DF2EE20EDE520F2EE2E2E2E000ACAE211
:10218F00E8F2E0EDF6E8FF20D2D3212020000AC6C6
:10219F00E4E0EB20EAE2E8F2E0EDF6E8FE20D2D34D
:1021AF002C20E020F2F3F220F7F2EE2DF2EE20E4F5
:1021BF00EBE8EDEDEEE52E2E2E2020000ACDE5F218
:1021CF0020E8EDF4EEF0ECE0F6E8E8212020000A3C
:1021DF00CFF0E8B8EC20E7E0EFF0EEF1E0202000E0
:1021EF000ACDE0F7E0EBEE20EFF0E8B8ECE0000A04
:1021FF00C8F1F2E5EAEBEE20E2F0E5ECFF20EEE6C7
:10220F00E8E4E0EDE8FF20EEF2E2E5F2E0000AC7D5
:10221F00E0EFF0EEF120E3F0F3EFEFFB20D2C8D2C6
:10222F00200020EEF220CACF20000A000ACEF2EFE3
:10223F00F0E0E2EAE020CED220EDE020CACF20008D
:10224F00202020CFEEE2F2EEF020EAEEECE0EDE41B
:10225F00FB0A00FF1E6FFF1E74FF1E7CFF1E84FF14
:10226F001E8EFF1E96FF1E9DFF1EA2FF1EA8FF1EA5
:04227F00AFFF1EB6D9
:103D160052668D0000000000000000000000000058
:103D2600000000000060A06A6500050002000005B2
:103D36000002000005000200000500020000050068
:103D46000200000500020000050002000005000256
:103D56000000050002000005000200000500020048
:103D66000005000200000500020000050002000038
:103D76000500020000050002000005000200000523
:103D86000002000005000200000500020000050018
:103D96000200000500020000050002000005000206
:103DA60000000500020000050002000005000200F8
:103DB60000050002000005000200000500020000E8
:093DC600050002000005000200E6
:0100320022AB
:0246F1008F51E7
:1046F300906B0AE0FF04F074BA2FF582E43467F597
:10470300837420F0E4FFEFC39D503BE55175F00344
:10471300A42462F582E43422F583E493FB740193C9
:10472300FA740293F98F827583001225F8FE906B59
:104733000AE024BAF582E43467F583EEF00F906B58
:064743000AE004F080C052
:01474900224D
:1049B900742D2FF582E43461F583E0FE64206016DE
:1049C900906B0AE0FD04F074BA2DF582E43467F5C2
:0649D90083EEF00F80DA0E
:0149DF0022B5
:1019EA00E4906B0AF0F548E54875F003A42462F523
:1019FA0082E43422F583E493FB740193FA7402932C
:101A0A00F91225DF7003021E6EE4F54AF54BF5491B
:101A1A00742D2549F582E43461F583E0FF700302F1
:101A2A001E69E54875F003A42462F582E43422F5C0
:101A3A0083E493FB740193FA740293F9854A8275DD
:101A4A0083001225F8FEEFB50608754B01054A0218
:101A5A001E64E54B7003021E64EE6003021E5FAD56
:101A6A004AAF481246F1E548B40A004003021E692B
:101A7A00901A81F8282873021A9F021B3D021B73D1
:101A8A00021B78021B7D021B84021B89021C660250
:101A9A001D49021E2CAF491249B9742D2549F9E492
:101AAA003461FA7B01C0031B8B54755500755600CF
:101ABA00E4F557D003122E748F508E4F8D4E8C4DF5
:101ACA00E4FFFEFDFCAB50AA4FA94EA84DC3122756
:101ADA00686022AB50AA4FA94EA84DE47F207E1C15
:101AEA00FDFC1226C812275A906B0EEEF0A3EFF0F7
:101AFA00E4906B0DF0E47FB07E04FDFCAB50AA4F7E
:101B0A00A94EA84DD31227685003021E69906B0D87
:101B1A007401F0AB50AA4FA94EA84D7F007EC2FDBA
:101B2A007C001226C812275A906B0EEEF0A3EFF033
:101B3A00021E69AF491249B9D20C742D2549F9E43C
:101B4A003461FA7B01C0031B8B547555007556002E
:101B5A00E4F557D003122E748F508E4F8D4E8C4D54
:101B6A00906720E550F0021E69D208021E69D2076A
:101B7A00021E69D208D207021E69D213021E69AF79
:101B8A00491249B9E4F54C742D2549F9E43461FA4E
:101B9A007B01C0031B8B54755500755600E4F5573D
:101BAA00D003122E748F508E4F8D4E8C4DE54C758E
:101BBA00F005A42465F9746A35F0FA7B01906B0686
:101BCA00EBF0A3EAF0A3E9F0E550122658742D25AC
:101BDA0049F582E43461F583E0FF642060047E0104
:101BEA0080027E00EF60047F0180027F00EF5E705A
:101BFA0003021E690549742D2549F582E43461F50D
:101C0A0083E0B42CC8054CE54CC394204003021E63
:101C1A00690549742D2549F9E43461FA7B01C00349
:101C2A001B8B54755500755600E4F557D003122ED8
:101C3A00748F508E4F8D4E8C4DE54C75F005A42453
:101C4A0065F9746A35F0FA7B01906B06EBF0A3EA4A
:101C5A00F0A3E9F0E550122658021BD7AF49124902
:101C6A00B9E4F54C742D2549F9E43461FA7B01C0D5
:101C7A00031B8B54755500755600E4F557D00312B3
:101C8A002E748F508E4F8D4E8C4DE54C75F005A4F9
:101C9A002465F9746A35F0FA7B01906B06EBF0A3C0
:101CAA00EAF0A3E9F0900001E55012266A742D25A6
:101CBA0049F582E43461F583E0FF642060047E0123
:101CCA0080027E00EF60047F0180027F00EF5E7079
:101CDA0003021E690549742D2549F582E43461F52C
:101CEA0083E0B42CC8054CE54CC394204003021E83
:101CFA00690549742D2549F9E43461FA7B01C00369
:101D0A001B8B54755500755600E4F557D003122EF7
:101D1A00748F508E4F8D4E8C4DE54C75F005A42472
:101D2A0065F9746A35F0FA7B01906B06EBF0A3EA69
:101D3A00F0A3E9F0900001E55012266A021CB7AF41
:101D4A00491249B9E4F54C742D2549F9E43461FA8C
:101D5A007B01C0031B8B54755500755600E4F5577B
:101D6A00D003122E748F508E4F8D4E8C4DE54C75CC
:101D7A00F005A42465F9746A35F0FA7B01906B06C4
:101D8A00EBF0A3EAF0A3E9F0900003E55012266A0B
:101D9A00742D2549F582E43461F583E0FF642060FF
:101DAA00047E0180027E00EF60047F0180027F00D2
:101DBA00EF5E7003021E690549742D2549F582E418
:101DCA003461F583E0B42CC8054CE54CC39420403B
:101DDA0003021E690549742D2549F9E43461FA7B29
:101DEA0001C0031B8B54755500755600E4F557D096
:101DFA0003122E748F508E4F8D4E8C4DE54C75F01C
:101E0A0005A42465F9746A35F0FA7B01906B06EB38
:101E1A00F0A3EAF0A3E9F0900003E55012266A0263
:101E2A001D9AAF491249B9742D2549F9E43461FA6A
:101E3A007B01C0031B8B54755500755600E4F5579A
:101E4A00D003122E748F508E4F8D4E8C4D9067B9E1
:101E5A00E550F0800AE4F54BF54A0549021A1A05DD
:041E6A00480219F120
:011E6E002251
:103482007BFF7A1E79B71222E5906B0DE0602FA3C5
:10349200E0FEA3E0FFC3E49FFFE49EFEAB07FAE475
:1034A200F9F8FF7EC27D01FC1226C88F518E508D25
:1034B2004F8C4E7BFF7A1E79D91222E5802F906BBA
:1034C2000EE0FEA3E0FFC3E49FFFE49EFEAB07FA1B
:1034D200E4F9F87F207E1CFDFC1226C88F518E5025
:1034E2008D4F8C4E7BFF7A1E79D91222E57BFF7AB3
:1034F2001F7917A208E433F54E1222E57BFF7A1FEB
:103502007936A207E433F54E1222E57BFF7A1F7962
:1035120057A20CE433F54E1222E5300C1F7BFF7AE2
:103522001F7981906720E075F00AA4FFAEF0E48F66
:10353200518E50F54FF54E1222E5801D7BFF7A1F0A
:1035420079AA906720E075F00AA4FFAEF0E48F51EB
:103552008E50F54FF54E1222E57BFF7A1F79D590FA
:1035620067B9E075F00AA4FFAEF0E48F518E50F512
:103572004FF54E1222E57BFF7A1F79FB1222E57B83
:10358200FF7A20792CA213E433F54E1222E5754E10
:1035920001754F677550217BFF7A2079551222E51C
:1035A200754E01754F687550BA7BFF7A20796A12A1
:1035B20022E5754E01754F6675509F7BFF7A207923
:0535C200861222E52243
:024384008D4862
:10438600AA06A907754B018A4C894DE4F549124ADC
:10439600658F4AE54A643C6030E54A642C602AAB86
:1043A6004BAA4CA94DE54A1226587401254DF54DE8
:1043B600E4354CF54C0549124A658F4AE54A643C9A
:1043C6006007E549C3954840D6E5497016AB4BAA48
:1043D6004CA94D74201226587401254DF54DE4352F
:1043E6004CF54CE549B5480C74FF254DF54D74FF69
:0E43F600354CF54CAB4BAA4CA94DE4122658A1
:014404002295
:1028A5007E207FA61241F6EF4E70037F01227E2027
:1028B5007FA91241F6EF4E700302294C12463B9058
:1028C5006B21122779E4FFFEFDFC906B21E0F8A354
:1028D500E0F9A3E0FAA3E0FBC31227686025906B3B
:1028E50021E0F8A3E0A3E0A3E0E47F207E1CFDFC4B
:1028F5001226C812275A906B0EEEF0A3EFF0E49063
:102905006B0DF0E47FB07E04FDFC906B21E0F8A335
:10291500E0F9A3E0FAA3E0FBD31227684038906BF7
:102925000D7401F0906B21E0F8A3E0A3E0A3E07F34
:10293500007EC27D017C001226C812275A906B0EBC
:10294500EEF0A3EFF0800F906B0E74FFF0A374B858
:10295500F0E4906B0DF07E207FAF1241F6EF4E60F4
:102965000C124A65EF24D024FF92088002C2087E2B
:10297500207FB51241F6EF4E600C124A65EF24D068
:1029850024FF92078002C2077E207FBB1241F6EF2B
:102995004E600C124A65EF24D024FF920C8002C2CF
:1029A5000C7E207FC11241F6EF4E601312463BE4C8
:1029B5007B0AFAF9F81226C8906720EFF08005E443
:1029C500906720F07E207FC71241F6EF4E6011120E
:1029D500463BE47B0AFAF9F81226C89067B9EFF08E
:1029E5009067B9E07003740AF07E207FCD1241F63E
:1029F500EF4E600C124A65EF24D024FF921380023B
:102A0500C213E4906B20F07E207FD31241F6EF4E87
:102A1500600B7E677F217D801243848023906B202D
:102A2500E0FF04F074212FF582E43467F583742008
:102A3500F0906B20E02421F582E43467F583E4F01F
:102A4500E4906B20F07E207FD91241F6EF4E600BAB
:102A55007E687FBA7D801243848023906B20E0FFDF
:102A650004F074BA2FF582E43468F5837420F0908D
:102A75006B20E024BAF582E43468F583E4F0E49051
:102A85006B20F07E207FDF1241F6EF4E600B7E66F5
:102A95007F9F7D801243848023906B20E0FF04F0AC
:102AA500749F2FF582E43466F5837420F0906B20D3
:0E2AB500E0249FF582E43466F583E4F07F00B0
:012AC30022F0
:10485B00301234E4906475F0906A63E0FD906476F6
:10486B00F090667AE0906477F0A37404F09069633B
:10487B00E0543FF063A20190647963A201AF05128B
:0A488B002B9FC2127F01227F002242
:102CAD00906B0E74FFF0A374B8F0E4906B0DF09080
:102CBD0067B97464F0E4906B0AF0C2101228A5EFA6
:102CCD0060061219EA022E70E4F547F546742125C7
:102CDD0046F582E43467F583E0FF6070E547C39401
:102CED00205069EFB42004054680E2E54775F005F4
:102CFD00A42465F9746A35F0FA906B067401F0A39B
:102D0D00EAF0A3E9F074212546F9E43467FA7B0172
:102D1D00C0031B8B54755500755600E4F557D00351
:102D2D00122E74906B06E0FBA3E0FAA3E0F9EF120C
:102D3D002658054774212546F582E43467F583E06E
:102D4D00FF64206088EF6085054680E8E5477005E3
:102D5D00D210022E70E4F547F54674BA2546F58279
:102D6D00E43468F583E0FF6073E547C39420506C4D
:102D7D00EFB42004054680E2E54775F005A424650F
:102D8D00F9746A35F0FA906B067401F0A3EAF0A3BA
:102D9D00E9F074BA2546F9E43468FA7B01C0031BE7
:102DAD008B54755500755600E4F557D003122E74EB
:102DBD00906B06E0FBA3E0FAA3E0F9900003EF129D
:102DCD00266A054774BA2546F582E43468F583E032
:102DDD00FF64206085EF6082054680E8E4F547F5E5
:102DED0046749F2546F582E43466F583E0FF6073F3
:102DFD00E547C39420506CEFB42004054680E2E50E
:102E0D004775F005A42465F9746A35F0FA906B06E0
:102E1D007401F0A3EAF0A3E9F0749F2546F9E434B8
:102E2D0066FA7B01C0031B8B54755500755600E483
:102E3D00F557D003122E74906B06E0FBA3E0FAA3B6
:102E4D00E0F9900001EF12266A0547749F2546F5BB
:102E5D0082E43466F583E0FF64206085EF608205CF
:062E6D004680E81245DD7D
:012E7300223C
:10481F007544C0C209C206E4F528C212C20FC20114
:10482F00D211F53AF53F906B0BF09067B8F030135B
:10483F001290671F7403F0D22F9067B9E09067B89A
:0C484F00F08005E490671FF012489522ED
:10440500AC07D227E4FE9067A1E0FD25E0F0EC3093
:10441500E709E04401F0A227B392270517E517B491
:10442500081C9067A1E0851682851583F00516E5C1
:104435001670020515906A64E004F0E4F517EC25A2
:10444500E0FC0EBE08C09067A1E0FF25E0F0A226C3
:10445500302701B350079067A1E04401F00517E547
:1044650017B4081C9067A1E0851682851583F005B1
:1044750016E51670020515906A64E004F0E4F51778
:014485002214
:0237D200AB0743
:1037D400E4FD200038906B05E0FF30E10A6402F05C
:1037E400906B09E06429F0906B05E0FF25E0F09010
:1037F4006B09E0FE30E707906B05E04401F0EE252D
:10380400E0906B09F0EB30E704E04401F00517E5C4
:103814001724F8601F1460468000EB30E70A431B4E
:1038240001A204B392048003531BFEE51B25E0F5BB
:103834001B0238B9EB30E70A431B01A204B392041C
:103844008003531BFE851482851383E51BF0051446
:10385400E51470020513906A63E004F080573005A4
:1038640026D20E300D1E906B05E0FF30E10A640293
:10387400F0906B09E06429F0906B09E0FF906B0510
:10388400E04FFF227F0022300413EB20E720D20513
:10389400E51BB42004D20D8015C20D8011EB30E776
:1038A4000DD205E51BB42004D20D8002C20DC20066
:1038B400D204E4F517EB25E0FB0DED640860030288
:0438C40037D67F0074
:0138C80022DD
:02474A00AB07BB
:10474C00E4906A64F075476975483B751569751690
:10475C00E3854882854783E044C0F0E4F517FAEA24
:10476C00C39B5018854882854783E0FFC2261244BC
:10477C00050548E548700205470A80E3D226E4FFA8
:09478C001244057515697516E368
:014795002201
:023E80008F466B
:103E8200300103023F2F74FC2546F54613131354E9
:103E92001FFF2546FFE433CF2402CF3400FEC3EFD9
:103EA2009414EE64809480401130230B7E207FE5D1
:103EB200E4FBFDFC1235C7D2112275490185154A72
:103EC20085164B906A64E0FBE4F0754763754879A8
:103ED2007515677516A3854882854783E044C0F04F
:103EE20085174CE4F517FAEAC395465018854882BF
:103EF200854783E0FFC2261244050548E548700263
:103F020005470A80E2D226E4FF124405D201906AF4
:103F120064E09067B7F0906A64EBF0854A15854BD0
:0D3F220016751801751967751AA3854C17DF
:013F2F00226F
:103B6D00E4FF0F2405F582E43461F5837405F00F4D
:103B7D0074052401F582E43461F583E4F0754601A2
:103B8D00754766754892FEAB46E5481548AA4770DD
:103B9D00021547F91225DFFDAC070F74052CF582D0
:103BAD00E43461F583EDF00EBE04DC754601754716
:103BBD0066754896E4FEAB46E5481548AA4770027F
:103BCD001547F91225DFFDAC070F74052CF582E4BE
:103BDD003461F583EDF00EBE04DC75460175476664
:103BED0075489AE4FEAB46E5481548AA477002159C
:103BFD0047F91225DFFDAC070F74052CF582E4346F
:103C0D0061F583EDF00EBE04DC75460175476675F2
:103C1D00489EE4FEAB46E5481548AA477002154795
:103C2D00F91225DFFDAC070F74052CF582E4346124
:083C3D00F583EDF00EBE04DC7E
:013C4500225C
:10090E0030092DC3E5279543FFE5269542FED3EF2B
:10091E009440EE940040197B087D40AF43AE4212E6
:10092E003A92E5432440FFE43542540FF5428F439B
:10093E00201903020F6230180AC2189067B8E060DF
:10094E000214F090671FE0B40700501C900961F884
:10095E0028287302097C020A44020A44020B41024F
:10096E000DB7020B41020F37E490671FF0223013D0
:10097E001390671F7403F0D22F9067B9E09067B899
:10098E00F0D20A22200103020A3D9067B7E0906A76
:10099E0064F0C201D214E4F546906A64E0FFE546C5
:1009AE00C39F5026AB18AA19A91A1225DFFE743B55
:1009BE002546F582E43469F583EEF07401251AF5C7
:1009CE001AE43519F519054680CF75156975163B6C
:1009DE008515118516128F10851682851583A3E055
:1009EE005478FF64706003BF382590671F7401F060
:1009FE009067A27406F0D203202303020F627E21B9
:100A0E007F10906A64E0FBAD16AC151235C722302C
:100A1E0023107E217F1E906A64E0FBAD16AC15128A
:100A2E0035C790671F7401F09067A27403F022908F
:100A3E00671F7404F022200F03020AF5E540653BA0
:100A4E00604DE54024085438FFE53B54386F600490
:100A5E007E0180027E00906A64E060047D01800267
:100A6E007D00EE5D7003020F62851682851583E0B0
:100A7E00FEE540131313541F2432F8A6068F4005CB
:100A8E0016E51670020515906A64E014F080B390B6
:100A9E0067A2E06406603F301404D211C21490665F
:100AAE0093E0FCA3E0FDA3E0FEA3E0FFE4FAF9F877
:100ABE00EF2401FFEA3EFEE93DFDE83CFC90669323
:100ACE00122779E4F528D20AD22FD2B19067B9E075
:100ADE009067B8F080069067B87441F0C20F9067C7
:100AEE00A2E090671FF02230B10B300C0890672007
:100AFE00E09067B8F0C2B1300C0C30B0099067B816
:100B0E00E06003020F62851682851583E0FFE540E3
:100B1E00131313541F2432F8A607E5402408543843
:100B2E00F5400516E51670020515906A64E014F09E
:100B3E00D20F22200603020D45E53F5438653A7068
:100B4E0003020F62E53A24085438F53A131313548E
:100B5E001F242AF8E690693AF0200512E0FF1237BA
:100B6E00D28F46906A63E0D3948040CD802A200DC8
:100B7E0003020C4C90671FE064036003020C4C9060
:100B8E00693AE0FF1237D28F46300EADC20EC20662
:100B9E00C205C20AE546603CC2123023107E217F98
:100BAE003C7C697D63906A63E0FB1235C790669763
:100BBE00E0FCA3E0FDA3E0FEA3E0FFE4FAF9F8EF0A
:100BCE002401FFEA3EFEE93DFDE83CFC90669712EB
:100BDE002779806490693BE0FF906963E06F600362
:100BEE00301342906A63E024FEF0D21230230F7E5F
:100BFE00217F4A7C697D63E02402FB1235C7906633
:100C0E008FE0FCA3E0FDA3E0FEA3E0FFE4FAF9F819
:100C1E00EF2401FFEA3EFEE93DFDE83CFC90668FC5
:100C2E0012277980133023107E217F5E7C697D63CD
:100C3E00906A63E0FB1235C7E490671FF02290675D
:100C4E001FE0B4031B3023107E217F6B7C697D6314
:100C5E00906A63E0FB1235C7E490671FF0020D3C0B
:100C6E00300338C203906A63E0C39403501DD2125E
:100C7E00E014F030230D7E217F8C7C697D63E0FBD8
:100C8E001235C7E490671FF0020D3C7E217F9D7CDC
:100C9E00697D63906A63E0FB1235C790693BE0FFA4
:100CAE00906963E06F601A3023107E217F5E7C694D
:100CBE007D63906A63E0FB1235C7E490671FF08096
:100CCE006D90693CE0FF906964E0B5071A3023101F
:100CDE007E217FCB7C697D63906A63E0FB1235C712
:100CEE00E490671FF080473023117E217FDE7C6900
:100CFE007D63906A63E014FB1235C7301307E490EE
:100D0E00671FF08029906963E090693BF0906964F9
:100D1E00E090693CF0906965E090693DF07F0312C8
:100D2E00474A90671F7401F09067A27403F0C20ED9
:100D3E00C206C205C20A22202F2E30230B7E217F2F
:100D4E00EFE4FBFDFC1235C7E49067B8F0D20690D5
:100D5E006A63F0906B09F0906B05F0D204F517D230
:100D6E0000751369751463229067B8E06003020F73
:100D7E006230230A7E217FFEFBFDFC1235C7906692
:100D8E009BE0FCA3E0FDA3E0FEA3E0FFE4FAF9F88C
:100D9E00EF2401FFEA3EFEE93DFDE83CFC90669B38
:100DAE00122779E490671FF022301006E490671F37
:100DBE00F022906B0BE004F0E0C394204002E4F0CC
:100DCE00906B0BE075F005A42465F9746A35F0FAA2
:100DDE007B01906B06EBF0A3EAF0A3E9F01225DF9E
:100DEE00FF7003020F2B906B06E0FBA3E0FAA3E06B
:100DFE00F990000274011226259000011225F8FECA
:100E0E009000021225F8C39E5003020ED3906B067B
:100E1E00E0FBA3E0FAA3E0F9900002E412266A9048
:100E2E00000474011226259000031225F8FE90008E
:100E3E00041225F8D39E4013906B06E0FBA3E0FA54
:100E4E00A3E0F9900004740112266A906B06E0FB91
:100E5E00A3E0FAA3E0F990693BEFF09000041225AD
:100E6E00F8441090693CF0E4A3F09067A27403F08C
:100E7E00FF12474A202303020F247E227F1D906B10
:100E8E0006E0A3E0FAA3E02404F9E43AFCAD017B0A
:100E9E00011235C77F1E124AC57E227F31906B0626
:100EAE00E0A3E0FAA3E0AC02FD7B011235C77F1E82
:100EBE00124AC57E227F397C697DE3906A64E0FB2D
:100ECE001235C78051906B06E0FBA3E0FAA3E0F960
:100EDE001225DF90693BF0A37450F0E4A3F0906705
:100EEE00A27405F07F0312474A30232A7E227F3BED
:100EFE00906B06E0A3E0FAA3E0AC02FD7B01123595
:100F0E00C77F1E124AC57E227F397C697DE3906AB7
:100F1E0064E0FB1235C790671F7401F022906B0BD3
:100F2E0074FFF0E490671FF0229067B8E0702530F0
:100F3E00230A7E227F4FFBFDFC1235C790671F747C
:100F4E0001F09067A27405F0851115851216906A4E
:040F5E0064E510F046
:010F6200226C
:0B4AD000301105C2117F01227F00227F
:034AE200C2AE223F
:10406800020F63E493A3F8E493A34003F68001F2FC
:1040780008DFF48029E493A3F85407240CC8C33359
:10408800C4540F4420C8834004F456800146F6DF28
:10409800E4800B0102040810204080903D10E47E6B
:1040A800019360BCA3FF543F30E509541FFEE4931D
:1040B800A360010ECF54C025E060A840B8E493A3E4
:1040C800FAE493A3F8E493A3C8C582C8CAC583CA0F
:1040D800F0A3C8C582C8CAC583CADFE9DEE780BEC7
:013DCF0000F3
:1025DF00BB010689828A83E0225002E722BBFE02FA
:0925EF00E32289828A83E493222D
:1025F800BB010CE58229F582E5833AF583E0225098
:1026080006E92582F8E622BBFE06E92582F8E222E1
:0D261800E58229F582E5833AF583E49322FB
:10262500BB010FF8E58229F582E5833AF583E028B9
:10263500F0225009C58229F8E58226F622BBFE095B
:10264500C58229F8E22582F222F8EA2583F583E995
:03265500932822A5
:10265800BB010689828A83F0225002F722BBFE0161
:02266800F3225B
:10266A00F8BB010DE58229F582E5833AF583E8F0A6
:10267A00225006E92582C8F622BBFE05E92582C852
:02268A00F2223A
:10268C0075F008758200EF2FFFEE33FECD33CDCC05
:10269C0033CCC58233C5829BED9AEC99E582984088
:1026AC000CF582EE9BFEED9AFDEC99FC0FD5F0D665
:1026BC00E4CEFBE4CDFAE4CCF9A88222B800C1B98F
:1026CC000059BA002DEC8BF084CFCECDFCE5F0CBCD
:1026DC00F97818EF2FFFEE33FEED33FDEC33FCEB06
:1026EC0033FB10D703994004EB99FB0FD8E5E4F9C1
:1026FC00FA227818EF2FFFEE33FEED33FDEC33FCAE
:10270C00C933C910D7059BE99A4007EC9BFCE99AA1
:10271C00F90FD8E0E4C9FAE4CCFB2275F010EF2FE6
:10272C00FFEE33FEED33FDCC33CCC833C810D707E6
:10273C009BEC9AE899400AED9BFDEC9AFCE899F821
:0E274C000FD5F0DAE4CDFBE4CCFAE4C8F922B4
:0E275A00C3E49FFFE49EFEE49DFDE49CFC2290
:10276800EB9FF5F0EA9E42F0E99D42F0E89C45F0C7
:01277800223E
:0C277900ECF0A3EDF0A3EEF0A3EFF022D3
:10278500A8828583F0D083D08212279C12279C12C1
:10279500279C12279CE473E493A3C583C5F0C583E6
:1027A500C8C582C8F0A3C583C5F0C583C8C582C89E
:0127B5002201
:10228300E55A244EF8E6055A22784B302D02784E53
:10229300E475F0011228050225DF2026EB7F2ED2FC
:1022A300268018EF540F2490D43440D4FF302A0BE7
:1022B300EF24BFB41A0050032461FFE55B600215ED
:1022C3005B055EE55E7002055D302D0D784BE475B0
:1022D300F001122805EF0226580247967403D22D07
:1022E3008003E4C22DF55A8B4B8A4C894DE4F55B90
:1022F300F55DF55EE55B60077F201222BE80F57514
:102303005CFFC227C226C228C229C22BC22CC22EFE
:1023130012228CFF700D302D057F001222CFAF5E8D
:10232300AE5D22B4255FC2D5C22A12228CFF24D00F
:10233300B40A00501A75F00A785B30D50508B6FF69
:102343000106C6A426F620D5047002D22980D9241A
:10235300CFB41A00EF5004C2E5D22A0224CFD22709
:1023630080C6D22680C0D22880BCD2D580BAD22BD8
:1023730080B47F201222BE2028077401B55B004081
:10238300F1122283FF1222BE0222F7D22ED22C8018
:1023930095122283FB122283FA122283F94A4B708D
:1023A3000679A07A257BFF20282EE55B602A7E0034
:1023B3008E827583001225F860060EEE655C70F060
:1023C300C2D5EBC0E0EAC0E0E9C0E0EE122516D0CA
:1023D300E0F9D0E0FAD0E0FB1225DFFF60AAEBC002
:1023E300E0EAC0E0E9C0E01222BED0E02401F9D067
:1023F300E03400FAD0E0FBE55C0460DCD55CD98016
:10240300877BFF7A257912D228809C791080027904
:1024130008C22CC22E8008D2D5790A8004790AC258
:10242300D5E55C047002F55CE4FAFDFEFF1222833D
:10243300FC7B08202713122283FD7B1030260A120F
:102443002283FE122283FF7B20EC3382D592D55068
:1024530013C3E43026069FFFE49EFEE42027039D7A
:10246300FDE49CFCE4CBF8C227EC700CCFCECDCCC2
:10247300E824F8F870F38017C3EF33FFEE33FEED73
:1024830033FDEC33FCEB33FB994002FB0FD8E9EB54
:10249300302705F8D0E0C448B227C0E00AEC4D4E1F
:1024A3004F78207B0070C2EAB55C0040BCC0E012EC
:1024B3002518D0F0D0E0202704C4C0E0C4B227C060
:1024C300F01222A7D0F0D5F0EB0222F712286423F2
:1024D3009453240E5823654C23614224124F241A2B
:0F24E30044241A49237A43242055240446240410
:1024F2004524044725C05023692D236D2E23902B9C
:10250200237123238E2025A92A232948000023880A
:102512003F3F3F00790AA2D5202914302B09B91078
:10252200020404B9080104A2D5202C02500104209F
:1025320028689228B55B005034C0E07F203029190A
:102542007F30A228722C722B500F12256FC228C224
:102552002CC22BC22E7F30800F302B03E9C0E01239
:1025620022BE302B03D0E0F9D0E0B55BCC302B1784
:102572007F30B9100C1222BE7F58302A077F788034
:1025820003B908031222BE3028057F2D0222BE7F26
:1025920020202EF87F2B202CF322922880CF286E29
:1025A200756C6C2900D2271222833027F8C2277853
:1025B2005B30D50108F60223292D504349581222D7
:1025C200832403B405004001E49025BB931222AF9B
:0D25D200743A1222AFD229755B0402240E68
:102E74008B518A528953E4F55DF55CF55BF55AF59F
:102E840058F559E555455645546012EBC0E0EAC083
:102E9400E0E9C0E0AB54AA55A956122815AB510578
:102EA40053E553AA527002055214F91225DFF55E58
:102EB400C394094007E55ED3940D40E1E55E6420C8
:102EC40060DBE55EB42D054359038016E55EB42B43
:102ED40005435901800C74FF2553F55374FF355293
:102EE400F552E55760046410703FAB51AA52A953E0
:102EF4001225DF64306009E557702E75570A802962
:102F04009000011225F8FF64786004EFB45813436D
:102F1400590175571074022553F553E43552F5528F
:102F24008007E5577003755708AB510553E553AA5D
:102F3400527002055214F91225DFF55EC394614004
:102F44000AE55ED3947A5003535EDF74D0255EF5B0
:102F54005EC3940A400CE55E9411406D74F9255EDD
:102F6400F55EE55ED395575060435901855D6285F2
:102F74005C61855B60855A5FAF577E00E4FCFDAB06
:102F84005DAA5CA95BA85A1227B6C8ECC8C9EDC9EA
:102F9400CAEECACBEFCBE4FCFDFEEB255EF55DEE9D
:102FA4003AF55CED39F55BEC38F55AAF5DAE5CADE6
:102FB4005BFCAB62AA61A960A85FD31227685003C7
:102FC400022F2D435904022F2DE55920E003E480FC
:102FD4002DE55545564554601EAB51E55324FFF984
:102FE400E55234FFFAEBC0E0EAC0E0E9C0E0AB54DC
:102FF400AA55A956122815E55930E20774FFFFFEB9
:10300400FDFC22E559AF5DAE5CAD5BAC5A30E1032B
:0430140002275A2213
:1027B600E88FF0A4CC8BF0A42CFCE98EF0A42CFCC2
:1027C6008AF0EDA42CFCEA8EF0A4CDA8F08BF0A440
:1027D6002DCC3825F0FDE98FF0A42CCD35F0FCEB9F
:1027E6008EF0A4FEA9F0EB8FF0A4CFC5F02ECD3964
:0F27F600FEE43CFCEAA42DCE35F0FDE43CFC22D1
:10280500FAE6FB0808E6F925F0F618E6CA3AF622D4
:10281500BB011A89828A83D0F0D0E0F8D0E0F9D0E4
:10282500E0FAD0E0FBE8C0E0C0F00228935016E9DA
:10283500F8D083D082D0E0F9D0E0FAD0E0FBC082B6
:10284500C08302288ABBFE16E9F8D083D082D0E087
:0F285500F9D0E0FAD0E0FBC082C08302289C22B9
:10286400D083D082F8E4937012740193700DA3A303
:1028740093F8740193F5828883E473740293686017
:06288400EFA3A3A380DF17
:09288A00EBF608EAF608E9F62273
:09289300EBF0A3EAF0A3E9F02246
:09289C00EBF208EAF208E9F2226D
:00000001FF
